:100000000F29A0008417800484138E010C1C8E001D
:10001000232003190A29232003190A2923200A2946
:10002000A000B3200C080D0403190A29042184132D
:100030002008800664001C281D288C0A03198D0FD7
:100040001A2880060A2920088E0601308C008D01AE
:10005000000820050E06031D08008C0A03198D0FE9
:1000600028280800910190009F1727308F0010303A
:10007000452003308F00E83045208F016430452053
:100080008F010A304520100850288E0011088D007D
:1000900010088C00E8200C08031D9F139F1B08000C
:1000A000303E9200220884000930930003105D2046
:1000B000920C930B572803145D2884139F1D6C2802
:1000C000000820041F1D200680008417000820045B
:1000D000031C20068000772800082004031C20064B
:1000E0001F192006800084172009800577281F0D1E
:1000F00006398C0080208D008C0A80200000D428D6
:1001000000308A000C08820701347534033415343A
:1001100000343C340C34D9348F0022088400200988
:10012000B42084138F0803190A29F03091000E08B7
:1001300080389000F03091030319910003198F0368
:1001400003190A29A328B72003010C1820088E1FC1
:1001500020088E0803190301900FB0288006972805
:10016000B12800009A28FF3A841780050A290D0853
:100170000C0403198C0A80300C1A8D060C198D069C
:100180008C188D060D0D8C0D8D0D0A298F018E009A
:10019000FF308E07031C8F07031C0A2903308D00D4
:1001A000DF30D420C8288D01E83E8C008D09FC305A
:1001B000031CDD288C070318DA288C0764008D0FD8
:1001C000DA280C18E3288C1CE7280000E728080030
:1001D00091019001103092000D0D900D910D0E08BF
:1001E00090020F08031C0F0F91020318FE280E083F
:1001F00090070F0803180F0F910703108C0D8D0D3A
:10020000920BEC280C080A298C098D098C0A031919
:100210008D0A0800831303138312640008008316F9
:100220008501083086008312061183160611831299
:10023000061083160610831286108316861005306A
:100240008312A2000830A00004309F00FE3051202D
:100250000130512003308F00E830C7200530A20064
:100260000830A00004309F00FE3051208030512023
:100270002D30512020305120533051206F305120EB
:100280006E30512061305120723051202030512089
:1002900052305120613051206E3051206730512052
:1002A0006530512072305120203051202D305120A6
:1002B0000630A2001030A00064308E000A308C207E
:1002C00032308E0005308C2046308E000A308C2073
:1002D00032308E0002308C2003308F00E830C7208F
:1002E0000530A2000830A00004309F00FE305120ED
:1002F00080305120693051206E30512063305120C0
:100300006830512065305120733051203A305120EF
:1003100020305120203051202030512020305120D9
:1003200020305120203051202030512020305120C9
:10033000203051200530A2000830A00004309F007A
:10034000FE305120C03051206330512065305120A3
:100350006E30512074305120693051206D30512061
:100360006530512074305120653051207230512059
:10037000733051203A30512020305120203051200C
:100380002030512020305120F0210530A2000830CB
:10039000A00004309F00FE305120873051202708F4
:1003A0009100260833202030512020305120203069
:1003B00051200530A2000830A00004309F00FE301C
:1003C0005120CC30512025089100240833202030C2
:1003D00051202030512020305120C4296300EE29C3
:1003E00001308C008D010630840004301020013073
:1003F0008C0006308400083001200C08A8000D088D
:10040000A90028088C0029088D000F308E008F016C
:10041000E820A6000D08A70028088C0029088D00F8
:1004200006308E008F01E820A4000D08A5000130E1
:04043000C6200800DA
:02400E00F53F7C
:00000001FF
